:020000040000FA
:04080000E4EF04F02D
:1008100003B23DEF04F0F2B458EF04F09EB060EF85
:1008200004F09EB268EF04F0F2A81AEF04F0F2B2FE
:100830001CEF04F0C2EF04F0CD90F29207BC078EDB
:10084000078C9EA029EF04F00101463F29EF04F038
:10085000472B07AE34EF04F0CECF4EF1CFCF4FF1A0
:1008600046C150F147C151F1CF6ACE6A0101466BD2
:10087000476B9E90CD80C2EF04F00392030103EE1C
:1008800000F080517F0BE92604C0EFFF802B8151DF
:10089000805D700BD8A48B8200008051815D700B4D
:1008A000D8A48B9281518019D8B40790C2EF04F07C
:1008B000F2940101383FC2EF04F0392BC2EF04F08B
:1008C0009E900101463FC2EF04F0472BC2EF04F0B7
:1008D0009E92C3CF48F1C4CF49F1C28207B485EFDD
:1008E00004F03AC13EF13BC13FF13CC140F13DC192
:1008F00041F14EC152F14FC153F150C154F151C1B8
:1009000055F148C14AF149C14BF10201002FC2EF34
:1009100004F03C0E006FD57ED5BE32D0D6CF3AF172
:10092000D7CF3BF138C13CF1E86AE8CF3DF1010196
:1009300047A7A6EF04F0079C079E0101000E4E6F2B
:10094000600E4F6F3D0E506F080E516F01013ABFA0
:10095000B6EF04F03B67B6EF04F03C67B6EF04F087
:100960003D67B6EF04F0F288BBEF04F0F2984E6BEF
:100970004F6B506B516BD76AD66A0101386B396B7C
:10098000C2EF04F002C0E0FF005001C0D8FF100029
:10099000A6B2C8EF04F00CC0A9FF0BC0A8FFA69E2A
:1009A000A69CA684F29E550EA76EAA0EA76EA682DE
:1009B000F28EA694A6B2DAEF04F01200A96EA69EFB
:1009C000A69CA680A8501200076A0F010E0EC16EE9
:1009D000800EC06E030EC26E0F01896A110E926EF8
:1009E000080E8A6EF10E936E8B6A800E946EF18EF5
:1009F0000F01280ED56EF28AB00ECD6E9D800101DA
:100A00004E6B4F6B506B516B526B536B546B556B02
:100A1000566B576B586B596B079C079E760ECA6EC8
:100A20009D8202013C0E006FCC6A240EAC6E040164
:100A3000806B816B0F01900EAB6E0F019D8A0301DD
:100A4000806B816B8A6B8B9207900001F28EF28C27
:100A500007B0EBEF0AF08B740301805181197F0B13
:100A6000D8B4EBEF0AF013EE00F081517F0BE126D2
:100A7000812BE7CFE8FFE00BD8B4EBEF0AF023EED1
:100A800082F08A51070BD926E7CFDFFF8A2BDF5090
:100A9000780AD8A4EBEF0AF007808251720AD8B422
:100AA000EFEF06F08251630AD8B42DEF09F08251BE
:100AB000690AD8B476EF05F082517A0AD8B489EF82
:100AC00006F062EF09F0040114EE00F080517F0B94
:100AD000E12682C4E7FF802B12000D0E826F63ECCB
:100AE00005F00A0E826F63EC05F012000401690E36
:100AF000826F63EC05F004012C0E826F63EC05F04D
:100B00000101030E006F000E016F000E026F000E58
:100B1000036F7AEC0DF020C182F40401300E8227BD
:100B200063EC05F021C182F40401300E822763ECEE
:100B300005F022C182F40401300E822763EC05F037
:100B400023C182F40401300E822763EC05F024C136
:100B500082F40401300E822763EC05F025C182F493
:100B60000401300E822763EC05F026C182F40401F3
:100B7000300E822763EC05F027C182F40401300EA9
:100B8000822763EC05F004012C0E826F63EC05F004
:100B90000101030E006F000E016F000E026F000EC8
:100BA000036F7AEC0DF020C182F40401300E82272D
:100BB00063EC05F021C182F40401300E822763EC5E
:100BC00005F022C182F40401300E822763EC05F0A7
:100BD00023C182F40401300E822763EC05F024C1A6
:100BE00082F40401300E822763EC05F025C182F403
:100BF0000401300E822763EC05F026C182F4040163
:100C0000300E822763EC05F027C182F40401300E18
:100C1000822763EC05F004012C0E826F63EC05F073
:100C200001010A0E006F000E016F000E026F000E30
:100C3000036F7AEC0DF020C182F40401300E82279C
:100C400063EC05F021C182F40401300E822763ECCD
:100C500005F022C182F40401300E822763EC05F016
:100C600023C182F40401300E822763EC05F024C115
:100C700082F40401300E822763EC05F025C182F472
:100C80000401300E822763EC05F026C182F40401D2
:100C9000300E822763EC05F027C182F40401300E88
:100CA000822763EC05F004012C0E826F63EC05F0E3
:100CB000200EF86EF76AF66A04010900F5CF82F497
:100CC00063EC05F00900F5CF82F463EC05F0090050
:100CD000F5CF82F463EC05F00900F5CF82F463EC04
:100CE00005F00900F5CF82F463EC05F00900F5CFBB
:100CF00082F463EC05F00900F5CF82F463EC05F0B3
:100D00000900F5CF82F463EC05F06DEC05F062EFBD
:100D100009F08351630AD8A462EF09F08451610A93
:100D2000D8A462EF09F085516C0AD8A462EF09F0EB
:100D30008651410A2EE08651440A07E08651420A54
:100D4000D8B4DCEF06F062EF09F00798079A0401C7
:100D50007A0E826F63EC05F00401780E826F63EC0B
:100D600005F00401640E826F63EC05F081A8C0EF0A
:100D700006F00401550E826F63EC05F0C5EF06F036
:100D800004014C0E826F63EC05F06DEC05F062EF30
:100D900009F00788079A04017A0E826F63EC05F068
:100DA0000401410E826F63EC05F00401610E826F55
:100DB00063EC05F0B6EF06F00798078A04017A0E97
:100DC000826F63EC05F00401420E826F63EC05F064
:100DD0000401610E826F63EC05F0B6EF06F00401CA
:100DE000720E826F63EC05F004012C0E826F63ECCF
:100DF00005F0078452C156F153C157F154C158F15F
:100E000055C159F13EC142F13FC143F140C144F1E6
:100E100041C145F14AC14CF14BC14DF1079401016B
:100E2000620E046F010E056F000E066F000E076F55
:100E300056C100F157C101F158C102F159C103F186
:100E4000E0EC0CF003BF6CEF07F00E0EDEEC04F0EC
:100E5000E8CF0CF10F0EDEEC04F0E8CF0DF1100E30
:100E6000DEEC04F0E8CF0EF1110EDEEC04F0E8CF7A
:100E70000FF129EC0CF056C104F157C105F158C12E
:100E800006F159C107F1E0EC0CF00782EDEC0BF034
:100E900029EC0CF00792EDEC0BF056C100F157C1B4
:100EA00001F158C102F159C103F10792EDEC0BF0C9
:100EB000CC0E046FE00E056F870E066F050E076FF0
:100EC000E0EC0CF000C10CF101C10DF102C10EF11A
:100ED00003C10FF1A5EF07F00101800E006F1A0E9C
:100EE000016F060E026F000E036F42C104F143C191
:100EF00005F144C106F145C107F1E0EC0CF003AF88
:100F000086EF07F0B4EC0DF0B8EF07F00E0EDEEC54
:100F100004F0E8CF0CF10F0EDEEC04F0E8CF0DF199
:100F2000100EDEEC04F0E8CF0EF1110EDEEC04F052
:100F3000E8CF0FF142C100F143C101F144C102F118
:100F400045C103F10782EDEC0BF00CC100F10DC1BE
:100F500001F10EC102F10FC103F10101000E046F96
:100F6000000E056F010E066F000E076F0EEC0DF000
:100F70007AEC0DF01D67C2EF07F00401200E826FBE
:100F8000C5EF07F004012D0E826F63EC05F024C15C
:100F900082F40401300E822763EC05F025C182F44F
:100FA0000401300E822763EC05F004012E0E826FDF
:100FB00063EC05F026C182F40401300E822763EC55
:100FC00005F027C182F40401300E822763EC05F09E
:100FD00004016D0E826F63EC05F004012C0E826F2C
:100FE00063EC05F042C100F143C101F144C102F1DB
:100FF00045C103F101017AEC0DF01EC182F4040138
:10100000300E822763EC05F01FC182F40401300E1C
:10101000822763EC05F020C182F40401300E8227A0
:1010200063EC05F021C182F40401300E822763ECE9
:1010300005F022C182F40401300E822763EC05F032
:1010400023C182F40401300E822763EC05F024C131
:1010500082F40401300E822763EC05F025C182F48E
:101060000401300E822763EC05F026C182F40401EE
:10107000300E822763EC05F027C182F40401300EA4
:10108000822763EC05F00401480E826F63EC05F0E3
:1010900004017A0E826F63EC05F004012C0E826F5E
:1010A00063EC05F056C100F157C101F158C102F1DE
:1010B00059C103F101017AEC0DF01EC182F4040163
:1010C000300E822763EC05F01FC182F40401300E5C
:1010D000822763EC05F020C182F40401300E8227E0
:1010E00063EC05F021C182F40401300E822763EC29
:1010F00005F022C182F40401300E822763EC05F072
:1011000023C182F40401300E822763EC05F024C170
:1011100082F40401300E822763EC05F025C182F4CD
:101120000401300E822763EC05F026C182F404012D
:10113000300E822763EC05F027C182F40401300EE3
:10114000822763EC05F00401630E826F63EC05F007
:1011500004012C0E826F63EC05F056C100F157C1FB
:1011600001F158C102F159C103F101010A0E046FE6
:10117000000E056F000E066F000E076FEFEC0CF00F
:10118000000E046F120E056F000E066F000E076F43
:101190000EEC0DF07AEC0DF01EC182F40401300E5D
:1011A000822763EC05F01FC182F40401300E822710
:1011B00063EC05F020C182F40401300E822763EC59
:1011C00005F021C182F40401300E822763EC05F0A2
:1011D00022C182F40401300E822763EC05F023C1A2
:1011E00082F40401300E822763EC05F024C182F4FE
:1011F0000401300E822763EC05F004012E0E826F8D
:1012000063EC05F025C182F40401300E822763EC03
:1012100005F026C182F40401300E822763EC05F04C
:1012200027C182F40401300E822763EC05F004012B
:10123000730E826F63EC05F004012C0E826F63EC79
:1012400005F0B4EC0DF04CC100F14DC101F18BEC97
:101250000AF06DEC05F062EF09F00401630E826F95
:1012600063EC05F004012C0E826F63EC05F067EC73
:1012700009F004012C0E826F63EC05F0DAEC09F042
:1012800004012C0E826F63EC05F056EC0AF00401A9
:101290002C0E826F63EC05F00101F80E006FCD0E8D
:1012A000016F660E026F030E036F7CEC09F0040100
:1012B0002C0E826F63EC05F06CEC0AF06DEC05F01F
:1012C00062EF09F003018A6B0790EBEF0AF0D89008
:1012D0000E0EDEEC04F0E8CF00F10F0EDEEC04F0B1
:1012E000E8CF01F1100EDEEC04F0E8CF02F1110EB0
:1012F000DEEC04F0E8CF03F10101000E046F000EF4
:10130000056F010E066F000E076F0EEC0DF07AEC04
:101310000DF01EC182F40401300E822763EC05F04B
:101320001FC182F40401300E822763EC05F020C156
:1013300082F40401300E822763EC05F021C182F4AF
:101340000401300E822763EC05F022C182F404010F
:10135000300E822763EC05F023C182F40401300EC5
:10136000822763EC05F024C182F40401300E822749
:1013700063EC05F025C182F40401300E822763EC92
:1013800005F004012E0E826F63EC05F026C182F495
:101390000401300E822763EC05F027C182F40401BA
:1013A000300E822763EC05F004016D0E826F63EC52
:1013B00005F01200120EDEEC04F0E8CF00F1130E7F
:1013C000DEEC04F0E8CF01F1140EDEEC04F0E8CF1F
:1013D00002F1150EDEEC04F0E8CF03F101010A0E74
:1013E000046F000E056F000E066F000E076FEFEC26
:1013F0000CF0000E046F120E056F000E066F000E4B
:10140000076F0EEC0DF07AEC0DF01EC182F40401B2
:10141000300E822763EC05F01FC182F40401300E08
:10142000822763EC05F020C182F40401300E82278C
:1014300063EC05F021C182F40401300E822763ECD5
:1014400005F022C182F40401300E822763EC05F01E
:1014500023C182F40401300E822763EC05F024C11D
:1014600082F40401300E822763EC05F004012E0E95
:10147000826F63EC05F025C182F40401300E8227EF
:1014800063EC05F026C182F40401300E822763EC80
:1014900005F027C182F40401300E822763EC05F0C9
:1014A0000401730E826F63EC05F012000A0EDEEC8D
:1014B00004F0E8CF00F10B0EDEEC04F0E8CF01F110
:1014C0000C0EDEEC04F0E8CF02F10D0EDEEC04F0C1
:1014D000E8CF03F18BEF0AF0060EDEEC04F0E8CF64
:1014E00000F1070EDEEC04F0E8CF01F1080EDEECAF
:1014F00004F0E8CF02F1090EDEEC04F0E8CF03F1CE
:101500008BEF0AF00101B4EC0DF007844AC100F141
:101510004BC101F107940101E80E046F800E056FC5
:10152000000E066F000E076FEFEC0CF0000E046F5C
:10153000040E056F000E066F000E076F0EEC0DF027
:10154000880E046F130E056F000E066F000E076FF6
:10155000E0EC0CF00A0E046F000E056F000E066F33
:10156000000E076F0EEC0DF07AEC0DF001011D6717
:10157000BFEF0AF00401200E826FC2EF0AF00401EF
:101580002D0E826F63EC05F024C182F40401300E4D
:10159000822763EC05F025C182F40401300E822716
:1015A00063EC05F026C182F40401300E822763EC5F
:1015B00005F004012E0E826F63EC05F027C182F462
:1015C0000401300E822763EC05F00401430E826FA4
:1015D00063EC05F0120081A8A9EF0BF007A862EFF9
:1015E0000BF00101800E006F1A0E016F060E026FE4
:1015F000000E036F3EC104F13FC105F140C106F189
:1016000041C107F1E0EC0CF003BFA9EF0BF0E7ECF0
:101610000BF03EC100F13FC101F140C102F141C1F7
:1016200003F10782EDEC0BF00CC104F10DC105F1E3
:101630000EC106F10FC107F1F80E006FCD0E016F5C
:10164000660E026F030E036FE0EC0CF00E0E0C6ED4
:1016500000C10BF0C8EC04F00F0E0C6E01C10BF0D2
:10166000C8EC04F0100E0C6E02C10BF0C8EC04F0D4
:10167000110E0C6E03C10BF0C8EC04F007840101DD
:10168000B4EC0DF04AC100F14BC101F107940A0E10
:101690000C6E00C10BF0C8EC04F00B0E0C6E01C117
:1016A0000BF0C8EC04F00C0E0C6E02C10BF0C8EC91
:1016B00004F00D0E0C6E03C10BF0C8EC04F007989B
:1016C000A9EF0BF007AAA9EF0BF007840101B4EC16
:1016D0000DF04AC100F14BC101F10794060E0C6EEA
:1016E00000C10BF0C8EC04F0070E0C6E01C10BF04A
:1016F000C8EC04F0080E0C6E02C10BF0C8EC04F04C
:10170000090E0C6E03C10BF0C8EC04F0078452C143
:1017100000F153C101F154C102F155C103F1079425
:10172000120E0C6E00C10BF0C8EC04F0130E0C6E20
:1017300001C10BF0C8EC04F0140E0C6E02C10BF0EA
:10174000C8EC04F0150E0C6E03C10BF0C8EC04F0ED
:10175000079A0401805181197F0B0BE09EA809D0E4
:1017600014EE00F081517F0BE126E750812B0F0131
:10177000AD6E28EF05F00CC100F10DC101F10EC1F5
:1017800002F10FC103F1000E046F000E056F010E90
:10179000066F000E076F0EEC0DF01DA1E6EF0BF0CB
:1017A0001451D8B4E6EF0BF00CC100F10DC101F1FA
:1017B0000EC102F10FC103F1000E046F000E056FA0
:1017C0000A0E066F000E076F0EEC0DF012000101FD
:1017D0000C6B0D6B0E6B0F6B12000101005305E1DA
:1017E000015303E1025301E1002BB0EC0CF0B4EC27
:1017F0000DF02C51006F2D51016F420E046F4B0EF6
:10180000056F000E066F000E076FEFEC0CF000C1C5
:1018100004F101C105F102C106F103C107F10CC1D8
:1018200000F10DC101F10EC102F10FC103F107B2C8
:101830001EEF0CF0E4EC0CF020EF0CF0E0EC0CF000
:1018400000C10CF101C10DF102C10EF103C10FF194
:101850001200B4EC0DF04CC100F14DC101F1060EC7
:10186000DEEC04F0E8CF04F1070EDEEC04F0E8CF84
:1018700005F1080EDEEC04F0E8CF06F1090EDEEC0F
:1018800004F0E8CF07F1E0EC0CF000C118F101C161
:1018900019F102C11AF103C11BF1290E046F000EE8
:1018A000056F000E066F000E076FEFEC0CF0EE0EEA
:1018B000046F430E056F000E066F000E076FE4EC19
:1018C0000CF018C104F119C105F11AC106F11BC1D0
:1018D00007F1EFEC0CF000C110F101C111F102C1F0
:1018E00012F103C113F1120EDEEC04F0E8CF04F1A3
:1018F000130EDEEC04F0E8CF05F1140EDEEC04F07C
:10190000E8CF06F1150EDEEC04F0E8CF07F10D0E7E
:10191000006F000E016F000E026F000E036FEFEC00
:101920000CF0180E046F000E056F000E066F000E0F
:10193000076F0EEC0DF010C104F111C105F112C1D9
:1019400006F113C107F1E4EC0CF06A0E046F2A0EE5
:10195000056F000E066F000E076FE0EC0CF0120032
:10196000BF0EFA6E200E2D6F2C6BD890003701370A
:1019700002370337D8B0C1EF0CF02D2FB6EF0CF0C3
:101980002C072D070353D8B412000331070B80092D
:10199000326F03390F0B010F2C6F80EC5FF0336F48
:1019A0002C0580EC5FF0335D335F2C6B3233D8B0A5
:1019B0002C272C3332A9D6EF0CF033512C271200F0
:1019C000D9EC0DF0D8B0120003510719286F9CEC28
:1019D0000DF0D8900751031928AF800F1200286B23
:1019E000C0EC0DF0D8A0D6EC0DF0D8B01200ABECE6
:1019F0000DF0B4EC0DF01F0E296FECEC0DF00B3573
:101A0000D8B09CEC0DF0D8A00335D8B01200292F27
:101A1000FDEF0CF028B1C3EC0DF01200286B04515F
:101A20000511061107110008D8A0C0EC0DF0D8A0D0
:101A3000D6EC0DF0D8B01200086B096B0A6B0B6B7B
:101A4000ECEC0DF01F0E296FECEC0DF007510B5D67
:101A5000D8A437EF0DF006510A5DD8A437EF0DF08A
:101A60000551095DD8A437EF0DF00451085DD8A0E9
:101A70004AEF0DF00451085F0551D8A0053D095FFC
:101A80000651D8A0063D0A5F0751D8A0073D0B5F5D
:101A9000D8900081292F24EF0DF028B1C3EC0DF070
:101AA000286BC0EC0DF0D890F0EC0DF007510B5DF9
:101AB000D8A467EF0DF006510A5DD8A467EF0DF0CA
:101AC0000551095DD8A467EF0DF00451085DD8A059
:101AD00076EF0DF0003F76EF0DF0013F76EF0DF061
:101AE000023F76EF0DF0032BD8B4120028B1C3ECFF
:101AF0000DF012000101286BC0EC0DF0D8B01200FF
:101B0000F5EC0DF0200E296F00370137023703374F
:101B100011EE27F00A0E2A6FE7360A0EE75CD8B0FE
:101B2000E76EE5522A2F8CEF0DF0292F84EF0DF090
:101B300028B11D81D8901200045100270551D8B05A
:101B4000053D01270651D8B0063D02270751D8B000
:101B5000073D032712000051086F0151096F025120
:101B60000A6F03510B6F12000101006B016B026BD6
:101B7000036B12000101046B056B066B076B12000F
:101B80000335D8A012000351800B001F011F021F54
:101B9000031F003FD3EF0DF0013FD3EF0DF0023FE5
:101BA000D3EF0DF0032B282B032512000735D8A007
:101BB00012000751800B041F051F061F071F043F5B
:101BC000E9EF0DF0053FE9EF0DF0063FE9EF0DF00D
:101BD000072B282B07251200003701370237033760
:101BE000083709370A370B3712001D6B1E6B1F6B46
:101BF000206B216B226B236B246B256B266B276B71
:021C00001200D0
:10BF0000E844F926000C160C2B0C3F0C520C640C68
:10BF1000760C860C960CA50CB30CC10CCF0CDC0C6B
:06BF2000E80CF40C000C1B
:00000001FF
